:020000040000FA
:02000000DE29F7
:080008009818181218162C08B4
:10001000A0002D08A100A201A3010E280F28640052
:100020008C1A2B28FF30A207031CA307031CA00770
:10003000031CA107031C0800220F0D28230F0E2804
:10004000FA30A2000030A3000F28981818121816D2
:1000500064008C1E28281A080314D9290408640097
:100060000C1E2F2899000314D929A401A501B3124D
:10007000D421031C0800D33E0319B3162D3EC63EFF
:10008000031846280A3E031C38284D28F33E03185F
:100090003828063E031C38280A3EA2000430A3007C
:1000A000A20EA20DA40DA50DA30B5128A90303199F
:1000B0009A28D421031C0800C63E031863280A3E70
:1000C000031C9A284D28F33E03189A28063E031C69
:1000D0009A280A3E4D28A401A501B312D421031C7D
:1000E0000800D33E0319B3162D3EC63E03186E28F2
:1000F0000A3E031C6E28A2000310240DA000250D4B
:10010000A100200DA10DA4070318A10A2108A5072D
:10011000A40DA50D2208A4070318A50AA903031915
:100120009A28D421031C0800C63E03189A280A3EC8
:1001300003187B28B31EA128A409A509A40A031942
:10014000A50A24080314D929B31329080319B317DE
:100150001030A8000301A40DA50D03180130D12013
:100160002808031DAA280800B31329080319B31788
:100170000530A8002730A3001030CA200330A300A8
:10018000E830CA20A3016430CA20A3010A30CA2083
:100190002408D128A2002508A1002408A000A2213B
:1001A0002008A000A8030319B31329080319DB28AA
:1001B0002802031808002008031DB313B31B08000E
:1001C000303ED4290830A600A7003708840035083F
:1001D00033193321331D3521360884008417340840
:1001E0008004A001A10126080319D929B3182821E8
:1001F0003608840000083405FF3EA00DA10DB31C95
:100200002821A60BF6282708331859292008D929B0
:100210000830A60037088400350833193321331D10
:10022000352136088400841734098005260803190F
:10023000D9293318592136088400A10CA00C0008D4
:100240003404031C340680002821A60B1B29D9295D
:10025000370884003508800600002E292F29302910
:1002600031298006080080043829FF3A80053929A1
:10027000FF3A84178005D929A301A200FF30A20705
:10028000031CA307031CD9290330A100E6304A212F
:100290003E29A101FC3EA000A109031C5529FF3005
:1002A0000000A00703185029A0076400A10F4F29E0
:1002B0000800A201A3016029A10CA00CA20DA30DAE
:1002C000FF3E03185C292308A1002208A000D929B9
:1002D0000310A00DA10DFF3E031868292008D9299D
:1002E0000310A10CA00CFF3E031870292008D92987
:1002F000A101A301A20001308429A101A301A20050
:1003000004308429A2000530A80023082102031D1F
:100310008B2922082002043003180130031902300F
:100320002805031DFF30D929A2002008A6002408B3
:10033000A0002608A4002108A6002508A100260880
:10034000A500A429A501A4011030A600210DA40D2B
:10035000A50D2208A4022308031C230FA5020318DD
:10036000B8292208A40723080318230FA5070310A0
:10037000A00DA10DA60BA6292008D9291030A80090
:10038000A101A001A70CA60C031CCC292208A007E0
:1003900023080318230FA107A10CA00CA50CA40C83
:1003A000A80BC2292408D929840031088A00300802
:1003B00082008313031383126400080083168130C4
:1003C00099002430980083129030980083160730EB
:1003D0009F008117181583120830D2000130D30016
:1003E0000830C2000130C3000730CC000130CD001E
:1003F00083160610861406118611861306138612BC
:100400008312C401C501D001D101F90186138316FD
:10041000861383128612831686128312061383169E
:100420000613413083128A012F2054308A012F2075
:1004300034308A012F2035308A012F2078308A010C
:100440002F2078308A012F2078308A012F20203009
:100450008A012F2053308A012F2074308A012F20E7
:1004600061308A012F2072308A012F2074308A0176
:100470002F2069308A012F206E308A012F206730AB
:100480008A012F202E308A012F202E308A012F2022
:100490002E308A012F202E308A012F200D308A0124
:1004A0002F200A308A012F20BE01BF01EC01CA01B2
:1004B000CB01861583168611C83083128A013C2130
:1004C0008A110A1270238A110A12EB2D8A110A125C
:1004D000E02286118316861106308312B6000130A1
:1004E000B4000630B7000430B5000130B3006C082A
:1004F000A000A1018A0108214A08A0004B08A10020
:1005000010308A0109213808A0003908A1008A01A9
:10051000082164006C08683C8A110A120319972AA2
:1005200064006C08523C8A110A12031DAE2A063080
:10053000B6000130B4000630B7000430B500013019
:10054000B300A001A10110308A010921A001A1017D
:1005500010308A0109218A110A12CA2A64006C0823
:10056000563C8A110A120319BC2A64006C08543CD8
:100570008A110A12031DCA2A0630B6000130B400DF
:100580000630B7000430B5000130B300A001A1016E
:100590008A01082108003A08A0003B08A1003C0895
:1005A000A4003D08A5005308A30052088A01942125
:1005B000CE002108CF002408BE002508BF00080097
:1005C0000310CA0DCB0D39184A14391C4A103808CB
:1005D000B800B9010800F801F001861183168611F0
:1005E00006308312B6000130B4000630B700043084
:1005F000B5000130B3005730A000A1018A010821E5
:100600000630B6000230B4000630B7000430B50042
:100610000230B3008A01E220F6008A01E220F700EE
:10062000F80364007808003C8A110A120319202B91
:1006300064008A110A12F61F002B8A110A126B2B12
:1006400041308A012F2054308A012F2034308A0112
:100650002F2035308A012F2044308A012F2042304C
:100660008A012F2078308A012F2078308A012F20AC
:1006700078308A012F2020308A012F2042308A01D1
:100680002F2075308A012F2073308A012F20793076
:100690008A012F2020308A012F2045308A012F2007
:1006A00072308A012F2072308A012F206F308A0128
:1006B0002F2072308A012F2021308A012F200D3007
:1006C0008A012F200A308A012F200617831606136D
:1006D00083120130F00086158316861183120800FC
:1006E00086158316861183125230EC00CA01CB01A5
:1006F000B801B9018A016622C601C7014608A000F7
:100700004708A100A3011F308A017A218A110A1229
:10071000031D9E2B0630B6000230B4000630B70031
:100720000430B5000230B3008A01E220EB00C60AB3
:100730000319C70A8A110A12031D7E2B8615831618
:10074000861183120800D001D1018A01EB223C30CE
:100750007605C000C10101307605F4004008A00014
:100760004108A10002308A017321C0002108C100A4
:10077000A001A1014108A30040088A0182218A1139
:100780000A12031D0E2C44308A012F2061308A0189
:100790002F2074308A012F2061308A012F204630AB
:1007A0008A012F206C308A012F2061308A012F208E
:1007B00073308A012F2068308A012F2020308A016F
:1007C0002F2053308A012F2069308A012F207A3060
:1007D0008A012F2065308A012F203D308A012F2089
:1007E00035308A012F2031308A012F2032308A01A2
:1007F0002F206B308A012F2062308A012F20693030
:100800008A012F2074308A012F200D308A012F2079
:100810000A308A012F208A110A12DD2D0730A0002C
:10082000A1014108A30040088A0182218A110A120D
:10083000031D3B2C0430F10064007408003C8A1155
:100840000A12031D322C0830D2000130D3000830C8
:10085000C2000130C3000730CC000130CD008A1146
:100860000A123B2CD2010130D300C2010130C30077
:10087000FF30CC00CD010930A000A1014108A30048
:1008800040088A0182218A110A12031D682C08304F
:10089000F10064007408003C8A110A12031D5F2CE9
:1008A0000830D2000130D3000830C2000130C3004C
:1008B0000730CC000130CD008A110A12682CD20119
:1008C0000130D300C2010130C300FF30CC00CD01A4
:1008D0000D30A000A1014108A30040088A01822137
:1008E0008A110A12031D962C2030F100640074084E
:1008F000003C8A110A12031D8C2C1030D2000230E9
:10090000D3001030C2000230C3000F30CC000230E0
:10091000CD008A110A12962CD2010230D300C201F6
:100920000230C300FF30CC000130CD007108A600BA
:10093000A7018030A200A3018A01BE21D6002508AC
:10094000D7005608A0005708A1005208A20053087B
:10095000A3008A01A221D6002108D7005608A600CC
:100960005708A700A2010430A3008A01BE21D000CD
:100970002508D10053308A012F2074308A012F209E
:1009800061308A012F2074308A012F2075308A014E
:100990002F2073308A012F2020308A012F204230EF
:1009A0008A012F2079308A012F2074308A012F206C
:1009B00065308A012F203D308A012F2020308A01A6
:1009C0002F20A9017608A400A5012E30B000B101A6
:1009D0008A01A4200D308A012F200A308A012F209D
:1009E00044308A012F2061308A012F2074308A011F
:1009F0002F2061308A012F2046308A012F206C3051
:100A00008A012F2061308A012F2073308A012F2024
:100A100068308A012F2020308A012F2053308A012C
:100A20002F2069308A012F207A308A012F206530EB
:100A30008A012F203D308A012F2020308A012F206B
:100A4000A9017108A400A5012E30B000B1018A01EE
:100A5000B4206D308A012F2062308A012F20693046
:100A60008A012F2074308A012F200D308A012F2017
:100A70000A308A012F2050308A012F2061308A01EC
:100A80002F2067308A012F2065308A012F202030E7
:100A90008A012F2053308A012F2069308A012F20AC
:100AA0007A308A012F2065308A012F203A308A015E
:100AB0002F2020308A012F20A9015208A4005308BA
:100AC000A5002E30B000B1018A01B42020308A0187
:100AD0002F2042308A012F2075308A012F20663066
:100AE0008A012F2066308A012F2065308A012F204D
:100AF00072308A012F2020308A012F2053308A0142
:100B00002F2069308A012F207A308A012F2065300A
:100B10008A012F203A308A012F2020308A012F208D
:100B2000A9014208A4004308A5002E30B000B1017D
:100B30008A01B4200D308A012F200A308A012F202B
:100B40004D308A012F2061308A012F2078308A01B0
:100B50002F2069308A012F206D308A012F207530B7
:100B60008A012F206D308A012F2020308A012F200A
:100B700050308A012F2061308A012F2067308A018E
:100B80002F2065308A012F2073308A012F203A30C0
:100B90008A012F2020308A012F20A9015008A400AB
:100BA0005108A5002E30B000B1018A01B4200D30EB
:100BB0008A012F200A308A012F2008006908EC00E2
:100BC0004E08CA004F08CB003E08B8003F08B900E5
:100BD0008A016622080041308A012F2074308A0180
:100BE0002F206D308A012F2065308A012F206C3034
:100BF0008A012F2020308A012F2041308A012F20A6
:100C000054308A012F2034308A012F2035308A0158
:100C10002F2044308A012F2042308A012F20783043
:100C20008A012F2078308A012F2078308A012F20E6
:100C300020308A012F2044308A012F2065308A011C
:100C40002F206D308A012F206F308A012F200D3028
:100C50008A012F200A308A012F203D308A012F205F
:100C60003D308A012F203D308A012F203D308A01FE
:100C70002F203D308A012F203D308A012F203D302A
:100C80008A012F203D308A012F203D308A012F20FC
:100C90003D308A012F203D308A012F203D308A01CE
:100CA0002F203D308A012F203D308A012F203D30FA
:100CB0008A012F203D308A012F203D308A012F20CC
:100CC0003D308A012F203D308A012F203D308A019E
:100CD0002F200D308A012F200A308A012F208A010F
:100CE000A3230D308A012F200A308A012F204130A2
:100CF0008A012F2074308A012F206D308A012F2025
:100D000065308A012F206C308A012F2020308A0123
:100D10002F2044308A012F2061308A012F20743027
:100D20008A012F2061308A012F2046308A012F202E
:100D30006C308A012F2061308A012F2073308A01A4
:100D40002F2068308A012F2020308A012F20443044
:100D50008A012F2065308A012F206D308A012F20D3
:100D60006F308A012F200D308A012F200A308A012E
:100D70002F2057308A012F2061308A012F206930BF
:100D80008A012F2074308A012F2069308A012F2098
:100D90006E308A012F2067308A012F2020308A018F
:100DA0002F2066308A012F206F308A012F20723069
:100DB0008A012F2020308A012F2064308A012F20C1
:100DC00061308A012F2074308A012F2061308A011E
:100DD0002F202E308A012F202E308A012F202E30F6
:100DE0008A012F202E308A012F200D308A012F20DA
:100DF0000A308A012F204F308A012F2070308A015B
:100E00002F2074308A012F2069308A012F206F3003
:100E10008A012F206E308A012F2073308A012F2003
:100E20003A308A012F200D308A012F200A308A01A2
:100E30002F2031308A012F2020308A012F202D30A1
:100E40008A012F2020308A012F2052308A012F2042
:100E500065308A012F2061308A012F2064308A0199
:100E60002F2020308A012F2066308A012F207230F7
:100E70008A012F206F308A012F206D308A012F20A8
:100E800020308A012F2061308A012F2064308A01AE
:100E90002F2064308A012F2072308A012F20653084
:100EA0008A012F2073308A012F2073308A012F206E
:100EB0000D308A012F200A308A012F2032308A011A
:100EC0002F2020308A012F202D308A012F20203022
:100ED0008A012F2057308A012F2072308A012F205B
:100EE00069308A012F2074308A012F2065308A01F1
:100EF0002F2020308A012F2074308A012F206F305C
:100F00008A012F2020308A012F2061308A012F2072
:100F100064308A012F2064308A012F2072308A01C8
:100F20002F2065308A012F2073308A012F207330E3
:100F30008A012F2020308A012F2065308A012F203E
:100F400072308A012F2061308A012F2073308A018C
:100F50002F2065308A012F2020308A012F20663013
:100F60008A012F2069308A012F2072308A012F20B8
:100F700073308A012F2074308A012F200D308A01AE
:100F80002F200A308A012F2033308A012F20203071
:100F90008A012F202D308A012F2020308A012F2016
:100FA00057308A012F2072308A012F2069308A0140
:100FB0002F2074308A012F2065308A012F202030A5
:100FC0008A012F2074308A012F206F308A012F2050
:100FD00020308A012F2061308A012F2064308A015D
:100FE0002F2064308A012F2072308A012F20653033
:100FF0008A012F2073308A012F2073308A012F201D
:1010000020308A012F206E308A012F206F308A0114
:101010002F2020308A012F2065308A012F20723046
:101020008A012F2061308A012F2073308A012F20FE
:1010300065308A012F200D308A012F200A308A0165
:101040002F2034308A012F2020308A012F202D308C
:101050008A012F2020308A012F2057308A012F202B
:1010600072308A012F2069308A012F2074308A0162
:101070002F2065308A012F202F308A012F205230F7
:101080008A012F2065308A012F2061308A012F20AC
:1010900064308A012F2020308A012F2054308A01A9
:1010A0002F2065308A012F2073308A012F20743061
:1010B0008A012F2020308A012F2061308A012F20C1
:1010C00074308A012F2020308A012F2061308A015C
:1010D0002F2064308A012F2064308A012F20723043
:1010E0008A012F2065308A012F2073308A012F203A
:1010F00073308A012F2020308A012F202A308A0164
:101100002F204E308A012F204F308A012F2054305B
:101110008A012F2045308A012F2020308A012F207C
:101120004F308A012F206E308A012F206C308A01C7
:101130002F2079308A012F2020308A012F2077300C
:101140008A012F206F308A012F2072308A012F20D0
:101150006B308A012F2073308A012F2020308A01C2
:101160002F2069308A012F2066308A012F202030FD
:101170008A012F2070308A012F2072308A012F209F
:1011800065308A012F2076308A012F2069308A014C
:101190002F206F308A012F2075308A012F20733065
:1011A0008A012F206C308A012F2079308A012F206C
:1011B00020308A012F2065308A012F2072308A0169
:1011C0002F2061308A012F2073308A012F20653053
:1011D0008A012F2064308A012F200D308A012F20B0
:1011E0000A308A012F2035308A012F2020308A01D1
:1011F0002F202D308A012F2020308A012F204530CA
:101200008A012F2072308A012F2061308A012F201D
:1012100073308A012F2065308A012F2020308A0107
:101220002F2070308A012F2061308A012F206730F3
:101230008A012F2065308A012F2020308A012F203B
:101240004E308A012F206F308A012F2074308A019E
:101250002F2020308A012F2066308A012F20753000
:101260008A012F206E308A012F2063308A012F20BF
:1012700074308A012F2069308A012F206F308A0153
:101280002F206E308A012F2061308A012F206C3090
:101290008A012F2020308A012F2061308A012F20DF
:1012A00073308A012F2020308A012F2079308A0163
:1012B0002F2065308A012F2074308A012F200D30B5
:1012C0008A012F200A308A012F2036308A012F20F0
:1012D00020308A012F202D308A012F2020308A01D2
:1012E0002F2045308A012F2072308A012F20613053
:1012F0008A012F2073308A012F2065308A012F2028
:1013000020308A012F2062308A012F206C308A0120
:101310002F206F308A012F2063308A012F206B30FD
:101320008A012F2020308A012F204E308A012F2061
:101330006F308A012F2074308A012F2020308A01DB
:101340002F2066308A012F2075308A012F206E30C1
:101350008A012F2063308A012F2074308A012F20C8
:1013600069308A012F206F308A012F206E308A0168
:101370002F2061308A012F206C308A012F202030ED
:101380008A012F2061308A012F2073308A012F209B
:1013900020308A012F2079308A012F2065308A0180
:1013A0002F2074308A012F200D308A012F200A301F
:1013B0008A012F2037308A012F2020308A012F20E8
:1013C0002D308A012F2020308A012F2045308A01BC
:1013D0002F2072308A012F2061308A012F20733034
:1013E0008A012F2065308A012F2020308A012F208A
:1013F00063308A012F2068308A012F2069308A01EA
:101400002F2070308A012F2020308A012F202D308C
:101410008A012F2020308A012F2045308A012F2079
:101420006E308A012F2074308A012F2065308A01A6
:101430002F2072308A012F203A308A012F2020304D
:101440008A012F207E308A012F2037308A012F20F9
:1014500030308A012F2030308A012F2030308A012D
:101460002F2030308A012F2030308A012F20303059
:101470008A012F2030308A012F2030308A012F201E
:101480000D308A012F200A308A012F200D308A0169
:101490002F200A308A012F2041308A012F2064300A
:1014A0008A012F2064308A012F2072308A012F2078
:1014B00065308A012F2073308A012F2073308A0112
:1014C0002F2020308A012F206D308A012F20753087
:1014D0008A012F2073308A012F2074308A012F2037
:1014E00020308A012F2062308A012F2065308A0146
:1014F0002F2020308A012F2061308A012F202030B8
:101500008A012F2064308A012F206F308A012F201A
:1015100075308A012F2062308A012F206C308A01B9
:101520002F2065308A012F2020308A012F2077302C
:101530008A012F206F308A012F2072308A012F20DC
:1015400064308A012F2020308A012F2069308A01DF
:101550002F206E308A012F2020308A012F20683002
:101560008A012F2065308A012F2078308A012F20B0
:101570000D308A012F200A308A012F2054308A0131
:101580002F2068308A012F2065308A012F202030DB
:101590008A012F207E308A012F2020308A012F20BF
:1015A00028308A012F2074308A012F2069308A0167
:1015B0002F206C308A012F2064308A012F20653063
:1015C0008A012F2029308A012F2020308A012F20E4
:1015D00069308A012F2073308A012F2020308A0140
:1015E0002F2075308A012F2073308A012F2065301B
:1015F0008A012F2064308A012F2020308A012F2079
:1016000061308A012F2073308A012F2020308A0117
:101610002F2061308A012F2020308A012F20733043
:101620008A012F2074308A012F2061308A012F20F7
:1016300072308A012F2074308A012F202F308A01C6
:101640002F2073308A012F2074308A012F206F30B1
:101650008A012F2070308A012F2020308A012F200C
:1016600063308A012F206F308A012F2064308A0175
:101670002F2065308A012F200D308A012F200A305B
:101680008A012F2066308A012F206F308A012F2097
:101690006C308A012F206C308A012F206F308A0134
:1016A0002F2077308A012F2065308A012F20643067
:1016B0008A012F2020308A012F2062308A012F20BA
:1016C00079308A012F2020308A012F2074308A013E
:1016D0002F2068308A012F2065308A012F2020308A
:1016E0008A012F206F308A012F2070308A012F202D
:1016F00074308A012F2069308A012F206F308A01CF
:101700002F206E308A012F2020308A012F20613057
:101710008A012F206E308A012F2064308A012F2009
:1017200020308A012F2074308A012F2068308A01EE
:101730002F2065308A012F2020308A012F20613030
:101740008A012F2064308A012F2064308A012F20E3
:1017500072308A012F2065308A012F2073308A0170
:101760002F2073308A012F200D308A012F200A305C
:101770008A012F2045308A012F2078308A012F20BE
:1017800061308A012F206D308A012F2070308A014C
:101790002F206C308A012F2065308A012F203A30AB
:1017A0008A012F2020308A012F207E308A012F20AD
:1017B00031308A012F2030308A012F2030308A01C9
:1017C0002F2030308A012F2034308A012F203230F0
:1017D0008A012F2030308A012F2030308A012F20BB
:1017E00030308A012F200D308A012F200A308A01E3
:1017F0002F2077308A012F2069308A012F206C300A
:101800008A012F206C308A012F2020308A012F205E
:1018100072308A012F2065308A012F2061308A01C1
:101820002F2064308A012F2020308A012F2064303D
:101830008A012F2061308A012F2074308A012F20E5
:1018400061308A012F2020308A012F2062308A01E6
:101850002F2065308A012F2067308A012F206930C0
:101860008A012F206E308A012F206E308A012F20AE
:1018700069308A012F206E308A012F2067308A015B
:101880002F2020308A012F2061308A012F207430D0
:101890008A012F2020308A012F2068308A012F20D2
:1018A00065308A012F2078308A012F2020308A016C
:1018B0002F2030308A012F2030308A012F20303005
:1018C0008A012F2034308A012F2032308A012F20C4
:1018D00030308A012F2030308A012F2030308A01A9
:1018E0002F200D308A012F200A308A012F208A01F3
:1018F00025207E3C8A150A12031D772C0130A90091
:101900002530B000B1018A016B20F2000430A9003B
:101910002530B000B1018A013520BA002508BB008E
:101920000430A9002530B000B1018A013520BC0087
:101930002508BD0064007208073C8A110A160319C5
:10194000C9298A01CB220A308A012F200D308A0151
:101950002F2050308A012F2061308A012F206730DC
:101960008A012F2065308A012F203A308A012F20EA
:10197000A9014E08A4004F08A5002E30B000B10107
:101980008A01B42020308A012F2041308A012F2083
:1019900064308A012F2064308A012F2072308A013E
:1019A0002F203A308A012F20A9013E08A4003F08C9
:1019B000A5002E30B000B1018A01B4200D308A019B
:1019C0002F200A308A012F2064007208013C8A15FA
:1019D0000A1203192F2D64007208023C8A150A129C
:1019E0000319F02D64007208033C8A150A120319CA
:1019F000F02D64007208043C8A150A120319CE2ED9
:101A00004F308A012F2070308A012F2074308A01D4
:101A10002F2069308A012F206F308A012F206E30ED
:101A20008A012F2020308A012F2045308A012F2063
:101A300072308A012F2072308A012F206F308A0184
:101A40002F2072308A012F2021308A012F200D3063
:101A50008A012F200A308A012F208A01712E5230EC
:101A6000EC004E08CA004F08CB003E08B8003F0803
:101A7000B9008A0166220D308A012F200A308A01BE
:101A80002F2050308A012F2061308A012F206730AB
:101A90008A012F2065308A012F203A308A012F20B9
:101AA000A9014E08A4004F08A5002E30B000B101D6
:101AB0008A01B4200D308A012F200A308A012F209C
:101AC0000130C600C7014608A0004708A10053081E
:101AD000A30052088A017A218A150A12031D992D42
:101AE0000630B6000230B4000630B7000430B5004E
:101AF0000230B3008A01E220EB00640080306B0208
:101B00008A150A12031C862D2E30EB00640020304B
:101B10006B028A150A1203188F2D2E30EB006B080A
:101B20008A012F20C60A0319C70A8A150A12031D43
:101B3000632D8615831686110D3083128A012F209E
:101B40000A308A012F204D308A012F206F308A0100
:101B50002F2072308A012F2065308A012F203F30DC
:101B60008A012F2020308A012F2031308A012F2036
:101B70003D308A012F2079308A012F2065308A017B
:101B80002F2073308A012F2020308A012F203230FD
:101B90008A012F203D308A012F206E308A012F20AC
:101BA0006F308A012F200D308A012F200A308A01E0
:101BB0002F200130A9002530B000B1018A016B202F
:101BC000EB0064006B08013C8A110A12031D712EA0
:101BD000CE0A0319CF0A8A150A122F2D8A01712EF7
:101BE000C401C50145308A012F206E308A012F20A3
:101BF00074308A012F2065308A012F2072308A01CB
:101C00002F2020308A012F2074308A012F20653048
:101C10008A012F2078308A012F2074308A012F20EA
:101C200020308A012F207E308A012F2020308A0127
:101C30002F2028308A012F2074308A012F2069300C
:101C40008A012F206C308A012F2064308A012F20D6
:101C500065308A012F2029308A012F2020308A0107
:101C60002F2074308A012F206F308A012F202030DE
:101C70008A012F2065308A012F206E308A012F20A3
:101C800064308A012F200D308A012F200A308A010A
:101C90002F208430EC003E08B8003F08B9008A01CC
:101CA000662241308A012F2064308A012F2064305F
:101CB0008A012F2072308A012F203A308A012F208A
:101CC000A9013E08A4003F08A5002E30B000B101D4
:101CD0008A01B4200D308A012F200A308A012F207A
:101CE000E830AC000330AD008A0104208A150A12E6
:101CF000031C702EEB006B08A00020308A017D21B0
:101D0000D6006B08A0007F308A017821D8005608E1
:101D100058048A150A12031D702E64006B087E3C5D
:101D20008A150A120319A62E0630B6000130B40037
:101D30000630B7000430B5000130B3006B08A000D6
:101D4000A1018A0108218A150A12702E86158316B0
:101D50008611640083127208023C8A150A12031D60
:101D6000B32E8330EC0064007208033C8A150A121B
:101D7000031DBC2E8830EC004E08CA004F08CB0073
:101D80008A01662286158316861183128A01EB2248
:101D900086158316861183128A01712E57308A01A7
:101DA0002F2072308A012F2069308A012F20743051
:101DB0008A012F2069308A012F206E308A012F205E
:101DC00067308A012F2020308A012F2073308A014A
:101DD0002F2061308A012F206D308A012F20703032
:101DE0008A012F206C308A012F2065308A012F2034
:101DF00020308A012F2074308A012F2065308A011B
:101E00002F2078308A012F2074308A012F20203033
:101E10008A012F2074308A012F206F308A012F20F1
:101E200020308A012F2042308A012F2075308A010C
:101E30002F2066308A012F2066308A012F206530DE
:101E40008A012F2072308A012F2020308A012F2012
:101E500031308A012F203A308A012F20A9014E0803
:101E6000A4004F08A5002E30B000B1018A01B420B3
:101E700020308A012F2061308A012F2074308A019E
:101E80002F2020308A012F2041308A012F206430FA
:101E90008A012F2064308A012F2072308A012F207E
:101EA00065308A012F2073308A012F2073308A0118
:101EB0002F203A308A012F20A9013E08A4003F08B4
:101EC000A5002E30B000B1018A01B4200D308A0186
:101ED0002F200A308A012F208430EC003E08B80001
:101EE0003F08B9008A0166223E30C800C901C60118
:101EF000C7014608A0004708A1004908A3004808F8
:101F00008A017A218A150A12031DF72F47088A15BC
:101F10000A12031DDE2F46083E3C8A150A12031CD6
:101F2000DE2F8A150A129827EB008A150A12DE2F77
:101F30000F308A0046089F3E03188A0A82005734F1
:101F400065346C3463346F346D346534213420343B
:101F5000543468346934733420346934733420342D
:101F600061346E342034413474346D3465346C34EF
:101F700020344134543434343534443442343034ED
:101F800078347834783420346D346234693474347D
:101F90002034643461347434613466346C346134B4
:101FA00073346834203438342034703469346E34F7
:101FB0002034633468346934703421340630B60018
:101FC0000130B4000630B7000430B5000130B30072
:101FD0006B08A000A1018A0108216B088A012F204B
:101FE000C60A0319C70A8A150A12031D792F861516
:101FF000831686110D3083128A012F200A308A0140
:102000002F2052308A012F2065308A012F20613025
:102010008A012F2064308A012F2069308A012F2005
:102020006E308A012F2067308A012F2020308A01EC
:102030002F2062308A012F2061308A012F206330E7
:102040008A012F206B308A012F2020308A012F2017
:1020500062308A012F2075308A012F2066308A0174
:102060002F2066308A012F2065308A012F207230A0
:102070008A012F202E308A012F202E308A012F2016
:102080002E308A012F200D308A012F200A308A013C
:102090002F205430EC003E08B8003F08B9008A01F8
:1020A0006622C601C7014608A0004708A1004908EA
:1020B000A30048088A017A218A110A16031D77288D
:1020C0000630B6000230B4000630B7000430B50068
:1020D0000230B3008A01E220EB006B088A012F2056
:1020E000C60A0319C70A8A110A16031D5328861542
:1020F000831686110D3083128A012F200A308A013F
:102100002F2045308A012F2072308A012F20613024
:102110008A012F2073308A012F2065308A012F20F9
:1021200020308A012F2026308A012F2020308A017A
:102130002F2077308A012F2072308A012F206930BA
:102140008A012F2074308A012F2065308A012F20C8
:1021500020308A012F2074308A012F206F308A01AD
:102160002F2020308A012F2044308A012F20613017
:102170008A012F2074308A012F2061308A012F209C
:1021800046308A012F206C308A012F2061308A016D
:102190002F2073308A012F2068308A012F202030B1
:1021A0008A012F2073308A012F2065308A012F2069
:1021B00063308A012F2074308A012F206F308A010A
:1021C0002F2072308A012F202E308A012F202E30AE
:1021D0008A012F202E308A012F200D308A012F20D6
:1021E0000A308A012F208330EC004E08CA004F08C5
:1021F000CB008A01662286158316861183128A0116
:10220000EB22861583168611831252308A012F2005
:1022100065308A012F2061308A012F2064308A01C5
:102220002F2069308A012F206E308A012F206730DD
:102230008A012F2020308A012F2062308A012F202E
:1022400061308A012F2063308A012F206B308A0190
:102250002F2020308A012F2044308A012F20613026
:102260008A012F2074308A012F2061308A012F20AB
:1022700046308A012F206C308A012F2061308A017C
:102280002F2073308A012F2068308A012F202030C0
:102290008A012F2073308A012F2065308A012F2078
:1022A00063308A012F2074308A012F206F308A0119
:1022B0002F2072308A012F202E308A012F202E30BD
:1022C0008A012F202E308A012F200D308A012F20E5
:1022D0000A308A012F205230EC004E08CA004F0805
:1022E000CB003E08B8003F08B9008A016622C6014B
:1022F000C7014608A0004708A1004908A3004808F4
:102300008A017A218A110A16031D9D290630B6001A
:102310000230B4000630B7000430B5000230B3001C
:102320008A01E220EB006B088A012F20C60A0319FC
:10233000C70A8A110A16031D792986158316861184
:102340000D3083128A012F200A308A012F20463057
:102350008A012F2069308A012F206E308A012F20B8
:1023600069308A012F2073308A012F2068308A015A
:102370002F2065308A012F2064308A012F200D30F4
:102380008A012F200A308A012F208A01712E08002D
:10239000080041308A012F2072308A012F206530D9
:1023A0008A012F2020308A012F2079308A012F20A6
:1023B0006F308A012F2075308A012F2020308A014A
:1023C0002F2041308A012F2042308A012F205330A4
:1023D0008A012F204F308A012F204C308A012F2074
:1023E00055308A012F2054308A012F2045308A0130
:1023F0002F204C308A012F2059308A012F20203085
:102400008A012F2073308A012F2075308A012F20F6
:1024100072308A012F2065308A012F203F308A01D7
:102420002F2020308A012F2031308A012F203D308B
:102430008A012F2079308A012F2065308A012F20D0
:1024400073308A012F2020308A012F2032308A01F8
:102450002F203D308A012F206E308A012F206F30CF
:102460008A012F200D308A012F200A308A012F2067
:1024700054308A012F2068308A012F2069308A0168
:102480002F2073308A012F2020308A012F206D30B9
:102490008A012F2061308A012F2079308A012F2074
:1024A00020308A012F2074308A012F2061308A0168
:1024B0002F206B308A012F2065308A012F20203099
:1024C0008A012F2033308A012F2030308A012F20BB
:1024D00020308A012F2074308A012F206F308A012A
:1024E0002F2020308A012F2038308A012F203030D1
:1024F0008A012F2020308A012F2073308A012F205B
:1025000065308A012F2063308A012F206F308A01C5
:102510002F206E308A012F2064308A012F207330E3
:102520008A012F200D308A012F200A308A012F20A6
:102530000130A9002530B000B1018A016B20EB0009
:1025400064006B08023C8A110A1603193E2B4530C1
:102550008A012F2072308A012F2061308A012F20BA
:1025600073308A012F2069308A012F206E308A0152
:102570002F2067308A012F202E308A012F202E3005
:102580008A012F202E308A012F200D308A012F2022
:102590000A308A012F208611831686110630831295
:1025A000B6000130B4000630B7000430B500013089
:1025B000B300C730A000A1018A0108219430A00017
:1025C000A1018A0108218030A000A1018A0108210F
:1025D0009A30A000A1018A01082186158316861170
:1025E0000A3083128A01492186118316861106302A
:1025F0008312B6000130B4000630B7000430B500D5
:102600000130B3005730A000A1018A010821063033
:10261000B6000230B4000630B7000430B500023016
:10262000B3008A01E220F6008A01E220F7002E3092
:102630008A012F2064008A110A16F61F072B8615BF
:1026400083168611453083128A012F2072308A0149
:102650002F2061308A012F2073308A012F206530AE
:102660008A012F2064308A012F2021308A012F20F7
:102670000D308A012F200A308A012F208A01712E05
:1026800064008A110A16402B63008A110A16442B33
:02400E00753FFC
:00000001FF
